:100000000C9446000C9463000C9463000C94630001
:100010000C9463000C9463000C9463000C946300D4
:100020000C9463000C9463000C9463000C946300C4
:100030000C9463000C9463000C9463000C947300A4
:100040000C9463000C9463000C9463000C946300A4
:100050000C9463000C9463000C9463000C94630094
:100060000C9463000C9463000C9463000C94630084
:100070000C9463000C9463000C9463000C94630074
:100080000C9463000C9463000C94630011241FBE55
:10009000CFEFD0E1DEBFCDBF11E0A0E0B1E0E0E501
:1000A000F1E000E00BBF02C007900D92A030B10755
:1000B000D9F711E0A0E0B1E001C01D92A230B10774
:1000C000E1F70C9496000C9400009C0112BE109273
:1000D00001011092000180910001909101018217AD
:1000E0009307C9F708951F920F920FB60F9211242C
:1000F0008F939F93809100019091010101969093BD
:100100000101809300019F918F910F900FBE0F907E
:100110001F90189586B7826086BF8DE083BF12BEA0
:1001200087B7826087BF8DE781BF0895CFEFD0E1A9
:10013000DEBFCDBF0E948A00789481E087BB11E0CA
:1001400080E092E00E94650088B3812788BBF8CFE9
:00000001FF
